:020000020000FC
:0200000006C038
:02000C00D1C061
:100026000FED0DBF00E002B903E309B906E003B91D
:10003600539A549A80D00FE007BB08BB0CE90BBD5E
:100046000FE30ABD09E00EBD00E00FBD00E409BFE5
:100056006627772788275527332744E678945ED086
:10006600053689F45FD0013311F4C09845C00233D8
:1000760011F4C19841C0033311F4C2983DC0043352
:10008600D9F5C39839C0013689F44CD0013311F43F
:10009600C09A32C0023311F4C19A2EC0033311F450
:1000A600C29A2AC0043341F5C39A26C0043719F40C
:1000B60009EC30D021C0033711F439D01DC0083601
:1000C60011F4346019C0033629F43B7F18B31F605E
:1000D60018BB12C0053721F4413071F04A950CC0A7
:1000E600043621F4473C41F0439506C0083721F415
:1000F6004FD0902FC39A00C0B2CF04E50BD005E6CF
:1001060009D003E707D004E705D00AE003D00DE0E5
:1001160001D0A5CF5D9BFECF0CB908955F9BFECFA6
:100126000CB108955F9BFECF0CB1F4DF089505E591
:10013600F1DFFDCF08950F931F9302E611E003D080
:100146001F910F910895E02FF12FC895002029F0F7
:100156005D9BFECF0CB83196F8CF089548616C6C64
:100166006F202D2057696C6C6B6F6D6D656E20620C
:1001760065696D2043686174206D69742064656DDE
:1001860020415454696E793233313321200A0D00EF
:100196001F93C4DF0F70000F102F110F110F100FD8
:1001A600BDDF0F70010F1F9108950F930FB70F93C7
:1001B6001F935395583CE9F45527639532FF08C0C1
:1001C600162F1F700FE0102708B3007F012B08BB06
:1001D600992311F09A9501C0C3986C3349F46627A8
:1001E60073957C3329F477278395883109F488271A
:1001F60031601F910F910FBF0F9118950F930FB795
:100206000F930CB187DF013311F4C19A03C0003399
:1002160009F4C1980F910FBF0F911895451709F46E
:04022600C398C39A1C
:00000001FF
